:10000000EDC700000C9416080C9416080C94160802
:100010000C9416080C9416080C9416080C941608E8
:100020000C9416080C9416080C9438210C94A721F3
:10003000FDC70000FBC70000F9C70000F7C70000BC
:10004000F5C700000C947C24F1C70000EFC7000046
:10005000EDC70000EBC70000E9C700000C94D923EE
:10006000E5C70000E3C70000E1C70000DFC70000EC
:10007000DDC70000DBC70000D9C70000D7C70000FC
:100080000C942324D3C70000D1C70000CFC70000C1
:10009000CDC70000CBC70000C9C70000C7C700001C
:1000A000C5C70000C3C70000C1C7000005A84CCDEC
:1000B000B2D44EB93836A9020C50B9918688083CA2
:1000C000A6AAAA2ABE000000803F0000000000701F
:1000D0000100C0000C00CAA77C0A42F55508534233
:1000E00048195EF551120030000000274500409489
:1000F0001C0014F3190504F111042004000004414C
:10010000100400040000104208015E14450F40F086
:1001100001005955551351555D0D8C927C0857556A
:10012000550D5E55550D51520C015E55550F5655E6
:10013000550F00A0000000A4000000C2280080A20B
:1001400028008062080040500D0000E318009C92D7
:10015000241F5F555D0D9C1445115F1425075F55E5
:1001600055115F5114015E54551D1F41101F40F47D
:100170004500100421071F41181D1F0441105EF0A7
:10018000041F9C10041F5E54450F5F9214035ED43D
:10019000451F5F92341B5655550D41F005011F0454
:1001A00021071F4208011FE4410F1743181D07C113
:1001B000090151564D1100F0450000F0010040F4D6
:1001C000010080100C0010044110904A001480F0CF
:1001D00090480064904A0064904C0064904D006424
:1001E000904F00C880F09035000F9041000F904D67
:1001F000000F80F09030000590470005901D00052D
:1002000090340005905300059023000590430005AD
:10021000905B0005E09073001990700019907400D5
:100220001990720019E0903700789036008C903564
:1002300000A0903400B4903300C8903200DC9031BC
:1002400000F09030000480F05155495400434F4E67
:1002500054494E5545000700000304000106000202
:10026000040002020402040404040404040204025C
:10027000020004020006010004030000070001065A
:100280000003040001020102020101020101010256
:100290000101020201020100040300060100007FC7
:1002A000001C1C0808000E700E1C0C0402041A66C8
:1002B0001E06020408142E5E0E00080814142E5F99
:1002C000001010142E2F280020202C2F2C2020006E
:1002D000282F2E141010006F2E14140808000E5E24
:1002E0002E14080402061E661A0402040C1C0E706A
:1002F0000E0008081C1C007F0010181C380738006E
:1003000020303C332C102000383D3A140810007D7A
:100310003A14140808000A7A3A14040402021A7AF9
:100320001A02020404143A7A0A00080814143A7DE6
:10033000001008143A3D380020102C333C302000C7
:100340003807381C18100308031E3F3F3F3F3F1E6D
:100350003C7EFFFFFFFFFF7E3C4E4557205245434A
:100360004F52442100C0F0384C6623F1F3730080F3
:10037000C06030F0F07000C0F07020F0F0702030FD
:10038000F0F0F00080E0F0D070700000000000009D
:10039000C0F03C0E070303C3FF3E00F0F0E000C0D6
:1003A000E0703080E0F0D07070000000F0F03010AD
:1003B00030300307060406030301000007070603A5
:1003C00007070006070300070703000006070300EE
:1003D00000030704040603030000000000030704F1
:1003E00004040603010000000007070701000000E5
:1003F00003070404060303000707010000000000D0
:10040000C0FEFEC6E2323E1C0000C0E0A0E0E000FC
:100410000080C060E0E0E0000080C06020F0FF3FAE
:1004200003C0E0E00080E0E0080CCCC662723E1C35
:100430000E0F03010001070E0C00070F09090C063F
:10044000060F0F0C060F0F00000F0F080C060F0F02
:1004500000404767343E1F0701000C0D0D000000EF
:10046000009064005090550014906400289055004E
:100470001490640014905500149064000A80F09069
:100480006A0050905E0014906A0028905E001490FC
:100490006A0014905E0014906A000A80F070FC8E6E
:1004A00083C1713F0E0000C0F93F07010080C0E228
:1004B000A3B1919F8E40C0828BC9793F06181C164C
:1004C00013F1FC1F1340C08C8FCB7931010078FCF5
:1004D0009E8BF9730200C1F1390D07030160F69F8D
:1004E00099FD670202808E9FD1793F0E004F424EE8
:1004F0002D5930372056455220302E313200C0C69B
:10050000CFDFFFFB73037CFEFFC7E3FF7F3E00FFEF
:10051000FFFF1B1B1B03000303FFFFFF0303000080
:1005200000000000000080808080000000000000CB
:1005300000000000000080E0F058AC56AB55AB5511
:1005400000FF0101010202040810608000003FFF6B
:10055000AA55AA55AA55AA55A85FAC5CAC5CAC5C80
:10056000AC5C0CCF3C0000000103060D1A152A25D7
:100570002A252A2522151209040201000000FFFF86
:1005800057AB57AB57AB57AB03FF808080000000E1
:10059000000000000000FFFF55AA55AA55AA55AA61
:1005A00000FF000000010102040830C000001F7FAE
:1005B000D5AA55AA55AA55AA54AF56AE56AE56AEB0
:1005C000562E86671E000000000103060D0A151254
:1005D00015121512110A09040201000000000000A2
:1005E000000000008080C0C0C0C08080800000008B
:1005F000000000000000C0F078AC56AB55AA55AA28
:1006000000FF000000010102040830C00000FFFFED
:1006100055AA55AA55AA55AA00FFFEAE56AE56AE2B
:1006200056AE5607FE001F17151215121512151299
:10063000101F171215121512151215101F009045D4
:10064000000A80F00000502050001408221C413E97
:100650003E476B6D6D413E001C1C001C3E7F4352AB
:1006600045444954005245434F524400535441526B
:10067000542047414D450000000000F0FCFCFC0008
:1006800000000000000000000000000000000080EA
:10069000C0E0F0F8783C1C1CFCFCF8F00000000006
:1006A0000000C0E0F0F87C3C1E0E0F070707070FA4
:1006B0000E00000000C0F8FCFC7C38383C1C1C1C00
:1006C0001C0C0C0C0C000000F8FCFCFC3C1C1C1C62
:1006D0001C1C1C3CFCF8F8F00000000000C0E0F01E
:1006E000F87C3C1E0E0F070707070F0E0080F0FF77
:1006F000FF3F0700000000000000000000000000B5
:10070000C0F0FC7E7F7F777130303038F8FFFFFF1C
:100710001F0000000000070F1F1F1C1C1C1C1C3C9E
:10072000FCFCF8F000000000E0FEFFFFEFE160706D
:100730007030383818180000000000E0FEFF7F77A6
:100740007070F8F8FCDCCE8F070703010000000092
:1007500000070F1F1F1C1C1C1C1C3CFCFCF8F0009D
:10076000007C7FFFFFE3E070707838381C1C1E0EA1
:100770000E0000F8FFFF7F0300000000000000E013
:10078000FCFF7F0F01000000307070F0E0E0E0F04F
:10079000F0787C3E1F0F070300000070FFFFFFE3AF
:1007A000E0E0707078383C1C0C0C00000000F0FE9B
:1007B000FF7F0700000000000001030F3FFFFEF86D
:1007C000600000307070F0E0E0E0F0F0787C3E1FF8
:1007D0000F0703000000504C41592054494D45007B
:1007E000504C415920434F554E54005D20005B0052
:1007F000424553542031302053434F524553002D2E
:10080000204C4153455253202D000046454252553D
:1008100041525920323031390050524F4752414DE8
:100820004D4544204259204F424F4E4F00005448FE
:1008300049532050524F4752414D20495300524591
:100840004C454153454420554E444552005448457B
:10085000204D4954204C4943454E53452E002120FC
:100860005741524E494E47202100005448452053DD
:10087000435245454E20464C49434B455253005642
:100880004552592052415049444C592E2049542038
:100890004D415900434155534520444953434F4D21
:1008A000464F525420414E44005452494747455206
:1008B000204550494C4550544943005345495A55E9
:1008C0005245532E204245204341524546554C2E19
:1008D000003E41555551653E50524553532020200E
:1008E000544F204143434550540000000000003E57
:1008F0005B4F5B3E3E6B4F6B3E1C3E7C3E1C183C90
:100900007E3C181C577D571C1C5E7F5E1C00183CEB
:100910001800FFE7C3E7FF0018241800FFE7DBE734
:10092000FF30483A060E2629792926407F0505071B
:10093000407F05253F5A3CE73C5A7F3E1C1C080877
:100940001C1C3E7F14227F22145F5F005F5F06093C
:100950007F017F006689956A606060606094A2FF95
:10096000A29408047E040810207E201008082A1C87
:1009700008081C2A08081E101010100C1E0C1E0C53
:1009800030383E3830060E3E0E06000000000000F3
:10099000005F00000007000700147F147F14242A62
:1009A0007F2A122313086462364956205000080734
:1009B0000300001C2241000041221C002A1C7F1C55
:1009C0002A08083E08080080703000080808080857
:1009D000000060600020100804023E5149453E00BE
:1009E000427F400072494949462141494D3318141C
:1009F000127F1027454545393C4A4949314121116B
:100A000009073649494936464949291E000014005C
:100A1000000040340000000814224114141414147F
:100A2000004122140802015909063E415D594E7CDD
:100A30001211127C7F494949363E414141227F4192
:100A400041413E7F494949417F090909013E4141F0
:100A500051737F0808087F00417F41002040413FDB
:100A6000017F081422417F404040407F021C027FEA
:100A70007F0408107F3E4141413E7F090909063E3F
:100A80004151215E7F09192946264949493203010E
:100A90007F01033F4040403F1F2040201F3F403820
:100AA000403F631408146303047804036159494DFB
:100AB00043007F4141410204081020004141417F31
:100AC00004020102044040404040000307080020A7
:100AD000545478407F2844443838444444283844A7
:100AE00044287F385454541800087E090218A4A4DE
:100AF0009C787F0804047800447D40002040403DFD
:100B0000007F1028440000417F40007C0478047876
:100B10007C080404783844444438FC182424181809
:100B2000242418FC7C080404084854545424040465
:100B30003F44243C4040207C1C2040201C3C403052
:100B4000403C44281028444C9090907C4464544C81
:100B500044000836410000007700000041360800DC
:100B600002010204023C2623263C1EA1A161123A86
:100B70004040207A385454555921555579412154D3
:100B8000547841215554784020545579400C1E52D8
:100B9000721239555555593954545459395554547C
:100BA000580000457C410002457D420001457C40E3
:100BB000F0292429F0F0282528F07C545545002000
:100BC00054547C547C0A097F49324949493232489D
:100BD000484832324A4848303A4141217A3A424004
:100BE0002078009DA0A07D39444444393D404040D8
:100BF0003D3C24FF2424487E4943662B2FFC2F2BA9
:100C0000FF0929F620C0887E090320545479410049
:100C100000447D413048484A32384040227A007AC8
:100C20000A0A727D0D19317D2629292F28262929A6
:100C3000292630484D4020380808080808080808C8
:100C4000382F10C8ACBA2F102834FA00007B0000EF
:100C500008142A142222142A14089500220095AAA6
:100C6000005500AAAA55AA55AA000000FF001010BE
:100C700010FF00141414FF001010FF00FF1010F0FC
:100C800010F0141414FC001414F700FF0000FF000F
:100C9000FF1414F404FC141417101F10101F101F5D
:100CA0001414141F00101010F0000000001F10108A
:100CB00010101F10101010F010000000FF10101086
:100CC000101010101010FF10000000FF140000FFA3
:100CD00000FF00001F10170000FC04F4141417108C
:100CE000171414F404F40000FF00F714141414147F
:100CF0001414F700F7141414171410101F101F14F5
:100D00001414F4141010F010F000001F101F000055
:100D1000001F14000000FC140000F010F01010FF81
:100D200010FF141414FF141010101F00000000F026
:100D300010FFFFFFFFFFF0F0F0F0F0FFFFFF0000FB
:100D4000000000FFFF0F0F0F0F0F38444438447CA2
:100D50002A2A3E147E02020606027E027E026355A5
:100D60004941633844443C04407E201E2006027EF4
:100D7000020299A5E7A5991C2A492A1C4C72017206
:100D80004C304A4D4D303048784830BC625A463D70
:100D90003E494949007E0101017E2A2A2A2A2A4425
:100DA000445F444440514A444040444A514000005A
:100DB000FF0103E080FF000008086B6B0836123665
:100DC0002436060F090F0600001818000000101046
:100DD000003040FF0101001F01011E00191D171204
:100DE000003C3C3C3C0000000000060115012601CF
:100DF00037014A015D01720188019F01B801D201EA
:100E0000EE010B022A024B026E029302BA02E402C6
:100E100010033F037003A403DC0317045504970475
:100E2000DD0427057505C80520067D06E00649078F
:100E3000B8072D08A9082D09B9094D0AEA0A900B2F
:100E4000400CFA0CC00D910E6F0F5A1053115B122B
:100E500072139A14D41520178018F519801B231DBE
:100E6000DE1EB420A622B524E4263429A72B402E6A
:100E70000031EA330037453ABC3D68414C456B4987
:100E8000C84D68524F57805C00621011121315163E
:100E900017181A1C1D1F21232527292C2E31343702
:100EA0003A3E4145494E52575C62686E757B838B72
:100EB000939CA5AFB9C4D0DCE9F70301D5F08D143C
:100EC000A1C881CFD9F1AF2000140213021202157C
:100ED000020702080204010101020100501017106C
:100EE0009812ED0FDF0FFE12BB17581771159F1EDA
:100EF000001FDC1A00000000240027002A002D003B
:100F0000300000000000250028002B002E003100DA
:100F1000040404040403040502020202040302029E
:100F2000020206060606060604040202020404047F
:100F300008020110408040102040804080080204D8
:100F4000018040201002011080102040402000004D
:100F5000000200090F0000030401000C0000000063
:100F600000000000000000000000000000080B006E
:100F70000202020000090400000102020000052430
:100F800000100105240101010424020605240600C5
:100F9000010705810310004009040100020A000056
:100FA000000705020240000007058302400000041C
:100FB00003090412010002EF0201404123368000C0
:100FC000010102030141726475696E6F204C4C434C
:100FD00000414241313330360000E72411241FBE66
:100FE000CFEFDAE0DEBFCDBF11E0A0E0B1E0E2E993
:100FF000F7E502C005900D92AA33B107D9F728E0B2
:10100000AAE3B1E001C01D92A532B207E1F717E0F3
:10101000CEEED7E004C02197FE010E94762BCD3E94
:10102000D107C9F70E941E250C94C72B0C94000011
:101030002091210830E0209530954091220850E021
:101040002423352390E02823392381E0232B09F43E
:1010500080E00895DC0177FF11C022273327261B8B
:10106000370B842F042E000C990B281739072CF40A
:10107000460F70E060E0141634F008951416ECF793
:1010800060347105D4F7A038B105B8F7362FFB01ED
:10109000E40FF11D47FDFA95E134F10514F040E449
:1010A000461B37709FEF032E01C0990F0A94EAF791
:1010B000430F631B710977FF02C0695F7F4F83E0B5
:1010C000759567958A95E1F7FB01F695FE2FEE275A
:1010D000F795E795EA0FFB1FE75EFB4F14166CF6DA
:1010E000483074F468E070E0641B710947FD739543
:1010F0002FEF30E002C0359527956A95E2F79223ED
:101100005081952B90834850E058FF4F9FEFE6CFDA
:101110000F9397FF0CC0EE27FF27E81BF90B4E1724
:101120001F0609F00CF47AC0480F90E080E077FFCA
:101130000FC0AA27BB27A61BB70BE22F022E000C5D
:10114000FF0BAE17BF070CF069C0260F70E060E020
:10115000442309F463C08038910509F45FC0121676
:101160000CF05CC0603471050CF058C0DC01A40FB9
:10117000B11DA138B10514F040E8481B562FFB0102
:10118000E20FF11D27FDFA95E134F10514F020E49A
:10119000261B57703FEF052E01C0330F0A94EAF764
:1011A000250F651B710977FF02C0695F7F4F53E010
:1011B000759567955A95E1F77695762F6627779519
:1011C0006795860F971F875E9B4F12163CF5283058
:1011D00074F4E8E0F0E0E21BF10927FDF3956FEF0E
:1011E00070E002C075956795EA95E2F73623011124
:1011F0000DC03095FC01B42F508153235193B15051
:10120000D9F7285080589F4F3FEFDFCFDC01742F74
:101210006C91632B6D937150D9F7F3CF0F910895B3
:1012200090E0E9E1F4E091119FEF8FEF91939193BA
:10123000919391938150D0F70895E1E0F0E010D0C0
:10124000319728F068517C4F8F4F9F4FF9CFAB01FA
:10125000FC0106D0641775078E079F07D0F3089529
:10126000A4E9B3E02FB7F8947D918D919C9166B578
:101270002FBFA89B05C06F3F18F47F5F8F4F9F4F14
:1012800022E0660F771F881F991F2A95D1F70895CE
:101290009091AD03911103C08FEF9FEF08954FB769
:1012A000F89422E02093E9005091F200252F30E0DD
:1012B0001216130614F421E030E0232B31F02898A5
:1012C00084E68093AC038091F100552339F030918E
:1012D000F200311103C06BE66093E8004FBF552365
:1012E000D9F290E008952FB7F89483E08093E90055
:1012F0009091E800892F807295FF04C03091F20030
:1013000080E4831B2FBF08958091A40381110DC039
:1013100022E02093A00334E03093A1031092A303B2
:101320001092A20341E04093A40380EA93E0089561
:10133000B0E0A0E0EEE9F9E00C94842B6C01B62E4D
:10134000A72E7A0180910C01882309F451C02091C5
:10135000AD03222309F44CC000919F0300FF05C098
:101360001091E00012601093E000E70110E00AEF36
:10137000209711F41123A9F1B6DF811104C00150A7
:10138000B9F15BDFF5CF8C171D0611F00CF08C2F37
:101390009FB7F89433E03093E9004091E80045FDB1
:1013A00002C09FBFE5CFC81BD109EB2DFA2DBE2E81
:1013B000AF2E815020F0A190A092F100F8CF112320
:1013C00029F07AE37093E80010E0EBCF5091E80049
:1013D00055FDE7CF6AE36093E80011E0209709F339
:1013E000F3CF5D98A4E6A0939E031E141F043CF067
:1013F000C1E0D0E0F601D383C283F12CE12CC70118
:10140000CDB7DEB7EAE00C94A02BA1E0B0E0EBE0B2
:10141000FAE00C948C2B6983DC01ED91FC91028045
:10142000F381E02D41E050E0BE016F5F7F4F0995F1
:101430002196E2E00C94A82B83E08093E9002091B0
:10144000F200222319F03AE33093E80008954BDFCD
:1014500090E00895FC018485958597FD05C02FEFE8
:101460003FEF35872487089513CF0895CF93DF93F7
:10147000EC018C859D8597FF03C00ADF9D878C87D3
:101480008C859D85DF91CF910895FC01848595859C
:1014900097FD0BC03FB7F89442E04093E90080917C
:1014A000F2003FBF90E0019608959FB7F89422E0C4
:1014B0002093E9008091F2009FBF90E00895409151
:1014C0009A0350919B0320919803309199034217FE
:1014D0005307B4F49091E8009570E1F33091E8007F
:1014E00032FD19C08093F10080919A0390919B0383
:1014F00001968F739927892B19F45EEF5093E800BA
:10150000A0919A03B0919B031196B0939B03A09373
:101510009A0381E0089580E00895EF92FF920F937F
:101520001F93CF93DF93F82E192FE62E042F81E01F
:10153000860F880FC4DF83E0C2DFCF2DD12FEC0EE2
:10154000FD2EF11CCE15DF0599F007FF0FC0FE013F
:101550008491B5DF182F80E0B2DF812321968111BD
:10156000F1CFCDB7DEB7E6E00C94A42B8881F1CFA4
:1015700081E0F7CFB0E0A0E0E0ECFAE00C94872B3C
:10158000D82E8A01EB017B01E40EF51ECE15DF0596
:1015900051F0D7FE0EC0FE01849191DF219681119A
:1015A000F5CF0FEF1FEFC801CDB7DEB7E7E00C9422
:1015B000A32B8881F2CFA1E0B0E0E1EEFAE00C9439
:1015C0008A2B82E0898342E450E06DE67FE080E888
:1015D000D1DF9ADEFC01028113810115110589F02A
:1015E000D801ED91FC910280F381E02DBE016F5F87
:1015F0007F4FC801099597FD04C0F801008511854A
:10160000ECCF89812196E4E00C94A62B615030F058
:101610002091F100FC0120830196F8CF289884E600
:101620008093AC030895282F30E0F901E25BF04F7E
:101630009491F901E15DF04F8491205F304FF90101
:101640002491222309F430C09923E9F091509F306E
:10165000D0F4E92FF0E0E15DF44F0C94762B5D0BB4
:10166000610B3E0B550B590B430B430B430B640BA8
:101670006A0B6E0B720B780B430B7C0B7091800026
:101680007F7770938000E22FF0E0EE0FFF1FEE5F98
:10169000F04FA591B491FFB7F8949C91611132C0BD
:1016A000809589238C93FFBF0895709180007F7D82
:1016B000E8CF70918000777FE4CFA4B5AF77A4BD69
:1016C000E2CFA4B5AF7DFBCF509190005F775093F0
:1016D0009000D9CF509190005F7DF9CF509190004C
:1016E000577FF5CF4091C0004F774093C000CBCFDC
:1016F0004091C0004F7DF9CF3091C200377F3093C9
:10170000C200C1CF892BCECFCF93DF9390E0FC01F5
:10171000E15DF04F2491805F904FFC01849188231C
:10172000C9F090E0880F991FFC01EC50F14FA59192
:10173000B491FC01EE5FF04FC591D49161110DC0E1
:101740009FB7F8946C91209562236C93788127233E
:1017500028839FBFDF91CF910895623051F49FB7E6
:10176000F8943C91422F409543234C935881252B6C
:10177000EFCF8FB7F894EC912E2B2C938FBFEACF3D
:101780001F93CF93DF93182FEB0161E0BDDF20970C
:1017900039F460E0812F47DFDF91CF911F910895E9
:1017A000CF3FD10511F461E0F5CFE12FF0E0E25B2E
:1017B000F04FE491E150EF3008F07CC0F0E0ED51E3
:1017C000F44F0C94762BF20BF70BFC0B060C100C61
:1017D0005A0C5A0C5A0C1A0C240C2E0C380C450CB2
:1017E0005A0C4D0C24B5206824BDC7BDD5CFD4B547
:1017F000D062D4BDC8BDD0CF809180008068809376
:101800008000D0938900C0938800C6CF10918000DB
:10181000106210938000D0938B00C0938A00BCCFDD
:10182000F0918000F860F0938000D0938D00C09319
:101830008C00B2CFE0919000E068E0939000D093EC
:101840009900C0939800A8CFB0919000B062B09377
:101850009000D0939B00C0939A009ECFA0919000DF
:10186000A860A0939000D0939D00C0939C0094CF5B
:101870006091C00060686093C0007091C0007F7B81
:101880007093C000C093CF0087CF4091C0004062EA
:101890004093C000C093D0007FCF8091C200886089
:1018A0008093C2002091C2002B7F2093C200C0937E
:1018B000D20072CFC038D1050CF075CF6ACFAB0122
:1018C000FC01CEDC41505109E109F10928F06851D1
:1018D0007C4F8F4F9F4FF6CFAB01FC01C1DC6417EB
:1018E00075078E079F07D0F308950895B0E0A0E034
:1018F000ECE7FCE00C94842B6C017B018B01040F62
:10190000151FEB015E01AE18BF08C017D10759F0D3
:101910006991D601ED91FC910190F081E02DC60115
:101920000995892B79F7C501CDB7DEB7EAE00C94AC
:10193000A02B8FB18095807F669B88601C9B846004
:10194000089583B7817F83BF23B7216023BF889524
:1019500033B73E7F33BF0895E0918A03F0918B0344
:101960009081809189038095892380830895E82F51
:10197000F0E0E654F14FE491E13019F0E33089F002
:10198000089520916F002D7F20936F008091850333
:10199000A0918603B09187039C91809589238C93B5
:1019A00008951092810380918203A0918303B091E6
:1019B0008403F2CFCF92DF92EF92FF920F931F93A7
:1019C000CF939091B2038917A8F567FD33C0E82F34
:1019D000F0E0E654F14FC491E62FF0E0603390F56B
:1019E000E657F14F049110E0F12CE12C60E074E235
:1019F00084EF90E0A70198010E94CD282150310981
:101A00004109510961E02115310581E0480751057F
:101A10006CF060E970ED83E090E0A70198010E940E
:101A2000CD28215031094109510963E0C13089F0C5
:101A3000C330F9F0CF911F910F91FF90EF90DF909D
:101A4000CF900895EE0FFF1FE657F24F05911491C6
:101A5000CBCF40918100487F462B4093810030934B
:101A600089002093880030916F00326030936F00BE
:101A7000E1CF80919100887F862B809391003093F5
:101A8000990020939800109377030093760311E058
:101A90001093810320917100226020937100CACFBE
:101AA000E091AE03F091AF03BF016F5F7F4F709382
:101AB000AF036093AE032491922F907F822F8F709B
:101AC000903811F454DFECCF903949F43296F0930A
:101AD000AF03E093AE03FB0164916CDFE1CF903E76
:101AE00049F4A091B003B091B103B093AF03A093B8
:101AF000AE03D6CF903F19F41092B303089597FD2B
:101B0000CFCF3296F093AF03E093AE03FB01449145
:101B1000A0917603B0917703322F242F0E941B29C6
:101B20006C507E4F8F4F9F4F28EE33E040E050E0E7
:101B30000E94F92820937D0330937E0340937F0316
:101B40005093800380917D0390917E03A0917F0349
:101B5000B0918003892B8A2B8B2B61F461E070E0BC
:101B600080E090E060937D0370937E0380937F0319
:101B70009093800308950F931F93CF93DF93209149
:101B8000B403222319F1162FEC018091B3038823AB
:101B900079F0009123080617C8F000E03091B203F5
:101BA000031720F4802FE3DE0F5FF8CF1092B3030A
:101BB00010932308D093B103C093B003D093AF0325
:101BC000C093AE036DDF41E04093B303DF91CF914B
:101BD0001F910F910895A9E0B0E0E1EFFDE00C94B2
:101BE0007C2BCF8210E0F801E60FF71FF7FDE8C06D
:101BF000603871050CF0E4C0DA01AE0DB11DB7FD1F
:101C0000DFC0403451050CF0DBC0DA0157FF04C0DF
:101C1000AA27BB27A41BB50BA770BB27FA0157FD4A
:101C20003796F595E795F595E795F595E79557FF7F
:101C300007C0319748E050E05A01AA1ABB0AD50103
:101C4000CE2CC694C694C694D12C5E2D577019F034
:101C50005FEFC51AD50AAF01261B370B5601AE0E32
:101C6000BF1EBC82AB82F695FE2FEE27F795E79557
:101C70003B016E0E7F1E860F971F6C01CE0EDF1E7E
:101C8000DA82C982F12CE12C8B819C818417950723
:101C900009F496C04830510509F492C04F3F9FEFB8
:101CA00059070CF464C02701460C571C1301E0E8E7
:101CB0002E0E311C2E0C3F1CA980BA80AE0CBF1C0E
:101CC000BE82AD82CB0197FD42C04F3F540709F45D
:101CD00073C0ED81FE81D4885901A80EB91EFF8121
:101CE000F13009F04CC0F501A490EA2D0A2E01C094
:101CF000EE0F0A94EAF7DE2AED81FE81D48A10976E
:101D000031F14730510519F1E8E0F0E04F018A1A4E
:101D10009B0AAD80BE80A418B508A20CB31CF501C7
:101D2000D488F901E80FF91FF987E887FF81F130BE
:101D3000A1F5E885F985C490EC2DF0E0082C02C0EF
:101D4000F595E7950A94E2F7DE2AF501D48A019623
:101D5000ED81FE813196FE83ED83FC01E61BF70BDE
:101D6000E017F10724F48038910509F0ACCF4F5FFC
:101D70005F4F200F311FF0E8EF0EF11C85CFF5010A
:101D8000A490EA2DF0E00A2E02C0EE0FFF1F0A9485
:101D9000E2F7E095F095DE22AFCFE885F985C490B3
:101DA000EC2DF0E0082C02C0F595E7950A94E2F7D7
:101DB000E095F095DE22C9CF109709F0A5CFC7CFE7
:101DC0002996E2E10C94982B60387105E8F44034D0
:101DD0005105D0F4342F369536953695A0E83A9FC4
:101DE000F0011124E60FF71FE80FF91F6489CA01FB
:101DF0008770992741E050E001C0440F8A95EAF7C7
:101E0000222319F0462B448B089540954623FBCF9F
:101E1000ADE0B0E0EEE0FFE00C947C2B6A30C1F462
:101E2000FC01EA5EFB4FDC01A85EBB4F5C9198E0D1
:101E3000599FC001112440815181840F951F9183C6
:101E4000808314971D921C922D96E2E10C94982B9E
:101E50006D30D1F39D878C878C5E9B4F9A838983ED
:101E6000FC01808091802C853D85285E3B4F3C8322
:101E70002B8330E8831691040CF06FC0AC85BD85D0
:101E8000AA5EBB4F6D907C9040E4641671040CF028
:101E900064C0EB81FC81408045E0C401449E800D1C
:101EA000911D1124181619060CF057C0242C312C42
:101EB000910153E0220F331F5A95E1F7260D371D8C
:101EC000121613060CF049C0649F50011124BE8203
:101ED000AD8210E000E0E0E0053039F0ED81FE81F8
:101EE000E651F74FE00FF11FE491530198E0592EAE
:101EF0002E2F30E038872F83E170E987F12CE12C19
:101F0000E414D0F46401CE0CDF1CDB86CA86D12C2D
:101F1000C12CC41468F4A6014A0D5B1D29856A858D
:101F20007B858C859D8550DF9FEFC91AD90AF1CF3B
:101F3000AFEFEA1AFA0AE4CFEF81F885F595E79555
:101F40005A94A20CB31C5110D3CF0F5F1F4F820CB9
:101F5000931C0630110509F0BECFAB81BC813C91CA
:101F6000432F50E0E981FA8180819181B6E03B9F67
:101F7000800D911D1124A981BA818D939C93EC85CC
:101F8000FD85E75EFB4F6081662309F45DCF7AEF44
:101F900074039001759F300D112420583F4F28176E
:101FA00039070CF051CFAC85BD85ED91FC911197AF
:101FB0000190F081E02D6AE0CD01099545CF809137
:101FC0007403833339F484E033D8882319F082E032
:101FD00090E0089581E090E008958EE598E0909378
:101FE0007303809372032FE12093710339E03093E0
:101FF000740341E040937503089584E090E090936A
:10200000700380936F0308959C0190913503953080
:102010006CF484E09802F0011124E45EFC4F3383F9
:102020002283718360839F5F909335030895CF93DC
:10203000DF93D0911B03D150D0931B032D2F2F5032
:10204000330BC90163E070E00E94632B8AE39AEAD4
:10205000A3EEBEEE04C0B695A795979587956A95B1
:10206000D2F7C82FC170C0931A036FEF70E08AE0F7
:1020700087DB6FEF70E083E083DB8FE7C89F802D05
:1020800011246FEF70E0681B710989E079DB81E052
:1020900090E0DD2311F090E080E0DF91CF91089592
:1020A00088E780931B030895E7EDF1E0938199237E
:1020B00031F08FEF890F83832281290F2283359698
:1020C00083E0E731F80790F30895FC012081318126
:1020D00084E0359527958A95E1F763816203A00135
:1020E000639F500D112493E0559547959A95E1F71C
:1020F000848130E18302C0011124840F951F08956B
:102100006FEF8AEC91E037CD0895FADF83E090E03D
:102110009093700380936F030895F2DF82E090E064
:102120009093700380936F030895EADF1092540335
:102130001092530384E090E0909319038093180366
:102140000895DEDF81E090E09093190380931803F7
:102150000895809100019AEA811195E5492F4095F3
:1021600029E134E0F9010024919341939193419343
:102170000394D1F731E083278093000108958F9273
:102180009F92AF92BF92CF92EF92FF920F931F93C5
:10219000CF93DF93EC015B014A01E02EAB014F5F6F
:1021A0005F4FBC016F5F7F4FC12C022F940185E010
:1021B00094E011DDCC24C3949401A501BE0185E017
:1021C00094E009DDDF91CF911F910F91FF90EF9087
:1021D000CF90BF90AF909F908F900895AF92BF9295
:1021E000CF92DF92EF92FF920F931F93CF936C01E8
:1021F0005B018A017901C0E04A30510594F0CA01BF
:102200006AE070E00E94632BAB01B501C901880F41
:10221000991F880F991FF601E81BF90BCF01DEDF2C
:10222000C82FC8016AE070E00E94632BAC0183E014
:10223000440F551F8A95E1F743565B4F08E028E0AD
:10224000B501C6018C0F911DC7FD9A9598DFEE0C64
:10225000EE0C8C2F8E19885FCF911F910F91FF90FC
:10226000EF90DF90CF90BF90AF900895E5E5F3E059
:1022700025E030E089E398E561917191629FA001CA
:10228000639F500D729F500D1124840F951F2E5F78
:102290003F4F2F31310581F70895ADE0B0E0E3E520
:1022A000F1E10C947C2B6A30C9F4FC01EA5EFB4F2F
:1022B000DC01A85EBB4F9C916081718156E0959FC7
:1022C000600D711D11247183608314971D921C92FF
:1022D00081E090E02D96E2E10C94982B20EE260F01
:1022E0002034B0F79D878C878C5E9B4F9E838D83B7
:1022F000FC01008111814C855D85485E5B4F5B87E9
:102300004A87003811050CF064C0AC85BD85AA5E13
:10231000BB4F8D919C919B838A83803491050CF0F7
:1023200058C0FA015081452E512C9801B5E05B9FB1
:10233000200D311D112437FD4CC0AA81BB8136E030
:10234000539FA00DB11D1124B7FD43C0EC85FD8541
:10235000E55EFB4F7080AC85BD85A65EBB4F6C9083
:1023600074E0679FF0011124E65BFF4F8590959024
:10237000A590B490513009F05EC026E0D22EF12C29
:10238000E12CD501C40181709927AA27BB2780FCC5
:1023900002C0761471F0262D892B8A2B8B2B09F421
:1023A000272D4A815B814E0D5F1DB8018C859D856F
:1023B0000BDDB694A794979487943FEFE31AF30A42
:1023C00056E0E516F104E9F6DA940F5F1F4FD110DD
:1023D000D6CFAA85BB852C91422F50E0ED81FE819E
:1023E00080819181B6E02B9F800D911D1124AD81DC
:1023F000BE818D939C93EC85FD85E75EFB4F30811C
:10240000332309F465CF7AEF74039001759F300D83
:10241000112420583F4F281739070CF059CFAC85AD
:10242000BD85ED91FC9111970190F081E02D6AE05E
:10243000CD0109954DCF180106E009830A811B8162
:1024400096E09C83D501C40181709927AA27BB27F8
:1024500080FC02C0761481F1892B8A2B8B2B31F101
:102460006F826101B101640D751DC616D70624F592
:102470007801E40CF51CF986E886780117FF02C0A4
:10248000F12CE12C488559854134510514F040E484
:1024900050E0E416F50664F42F81A701B6018C859F
:1024A0009D8592DCBFEFEB1AFB0AECCF7F82D9CF80
:1024B000EFEFCE1ADE0AD6CFB694A79497948794FE
:1024C000FC81F150FC83040D151DF111BBCF8981F6
:1024D00081508983240C351C8111B0CF7ACFEF92C3
:1024E000FF920F931F93CF93DF938C017B01D0E07A
:1024F000C0E0F701EC0FFD1F6491662331F0C801C5
:10250000CCDE892B11F02196F4CFCE01CDB7DEB70A
:10251000E6E00C94A42B90931A088093190870930A
:102520001C0860931B08BA0185E094E0D8CF089599
:102530006F927F928F929F92AF92BF92CF92EF92C3
:102540000F93CF93DF930E94100920911B0388E71C
:1025500090E0821B91096CE270E00E94632B3B01CA
:102560002EE1A22E25E0B22E3CE1832E912CD0E06C
:10257000C0E081E090E06C167D0611F090E080E014
:10258000C0901A03C89EA001C99E500D1124445F3B
:102590005F4FCC24C39490E2E92E08E19501B40189
:1025A00085E094E018DB219688E1880E911C80E696
:1025B000A80EB11CC330D105E1F688E0E82E00E298
:1025C0002EEF34E04CE250E064E470E085E094E00B
:1025D00002DB4DEE54E06AE370E080E190E09BDFC7
:1025E000DF91CF910F91EF90CF90BF90AF909F90E0
:1025F0008F907F906F90089550CE0895CF92EF9274
:102600000F93CF9380917503882389F00E9410095E
:1026100001E027E040E868E070E090E080E00E94A0
:10262000880810921F08109220081092750380915C
:102630007403833308F049C0E0917203F09173038F
:102640009F012F5F3F4F3093730320937203C49118
:10265000C11123C091E090931F089093200834E0AB
:10266000309371038A5F80937403833301F748EDDD
:1026700058E069E370E08DE090E04DDFCC24C39436
:1026800087E0E82E07E021ED38E048E350E060E322
:1026900070E085E094E09FDACACF2091710330E0CA
:1026A00030931A082093190890E090931C088093A7
:1026B0001B086C2F85E094E09FDF009171030A5F97
:1026C00000937103C1320CF4B2CFCF910F91EF9010
:1026D000CF9008951092B403E5E6F0E08081886021
:1026E00080830895E5E6F0E08081877F808321E0A4
:1026F0002093B403089580E80E941808882359F0B5
:1027000080913A0318163CF4815080933A036FEF9E
:102710008EE396E030DA80E10E9418088823B1F059
:1027200020913A03422F022E000C550B8091350365
:10273000082E000C990B0197481759073CF42F5F9E
:1027400020933A036FEF8EE396E015DA88E00E945B
:102750001808882331F02091B403211113C0C2DF7F
:10276000CFDC84E00E941808882359F0E0913A03F6
:1027700034E0E302D0011124A45EBC4FED91FC9142
:1027800009950895A7DFECCF089590E080E00895C3
:1027900097FF0BC022273327281B390B421713063C
:1027A00031F02CF0480F90E080E0411101C0089515
:1027B00060347105E0F7DC01A40FB11DA138B1054B
:1027C00014F040E8481B362F3770B1E001C0BB0F52
:1027D0003A95EAF7FB0133E0F595E7953A95E1F78D
:1027E000F695FE2FEE27F795E795E80FF91FE75EC0
:1027F000FB4F80818B2B81934150D9F70895B0E036
:10280000A0E0E5E0F4E10C94852B142FB22EC62F46
:10281000660FDD0B6E019FEFC91AD90AE82E880FEB
:10282000FF0800E0B601C70101960E948808412F09
:10283000BE01C701ADDFBE016B0D711DB7FC7A95FE
:1028400061507109412FC701A3DFBA94BA944B2D8F
:10285000B601C7010E942A08C701810F911D4B2DA7
:10286000B60101970E942A08CDB7DEB7E9E00C94C3
:10287000A12BB0E0A0E0EFE3F4E10C94842B2091D5
:1028800036032C5F409137034C5F609138036250F0
:10289000809139038250B3DF10E000E0B12CA12C0D
:1028A0009CE1C92E93E0D92EC09138030C2E000C68
:1028B000DD0BE09039030E2C000CFF0820913A0349
:1028C000A22F022E000CBB0B80913503082E000CAA
:1028D000990BA816B906DCF4F60142815381B801C0
:1028E0006C0F7D1FC7010C9624E030E0AA16BB06D2
:1028F00011F030E020E0821B930B0DDEFFEFAF1AEA
:10290000BF0A84E0C80ED11C0A5F1F4FCDCF16E06E
:10291000BE012102600D711D112401E025E045E09A
:10292000C7010E948808809137035701A80EB11C87
:1029300087FDBA94C0903603CC0DD11DC7FCDA9543
:102940002797B50165517109CC24C39487E0E82E1F
:102950000EE020E536E0AE0185E094E03CD9209120
:10296000B403129F900111242C5B394FB5016650BE
:10297000710906E0AE0185E094E02DD9CDB7DEB750
:10298000EAE00C94A02BA1E2B0E0E9ECF4E10C94B5
:10299000872B7C01FA01CB01D22E19A221E02D1543
:1029A00010F02AE0D22E8E010F5D1F4F2D2D30E04A
:1029B00050E040E0BF010E94F928F901CA016A30E5
:1029C000ECF4605DD8016E938D01232B242B252B15
:1029D00069F790E080E0109769F0FD010190002018
:1029E000E9F7AF01415051094A1B5B0BBD01C7011B
:1029F0000E94760CA196E7E00C94A32B695CE2CFD1
:102A0000B0E0A0E0E6E0F5E10C94862B8C016A01D1
:102A10007B01F7FE14C06DE2EFDDEC014427552782
:102A2000BA014C195D096E097F092AE0C801ABDFC4
:102A30008C0F9D1FCDB7DEB7E8E00C94A22B2AE0E7
:102A4000A2DFF8CF0E942C2829E130E040E050E0DE
:102A50000E94CD2888E0860F0895B0E0A0E0E3E36F
:102A6000F5E10C94862B7C01162F042FC0901703E0
:102A70000C2C000CDD080E942C2825E02C9DE00188
:102A80002D9DD00D1124C952DE4F20EA35E040E0E3
:102A900050E00E94CD28605D7240810991096E0D61
:102AA0007F1D7983688383E08A830E942C28212FED
:102AB00030E050E040E00E94CD28160F1B830C83CD
:102AC00080911703082E000C990B019660E470E0CA
:102AD0000E94632B80931703CDB7DEB7E8E00C9418
:102AE000A22BA6E0B0E0E7E7F5E10C947C2B31DB0C
:102AF0005BE3C52E53E0D52E10E0012F0170F601E7
:102B0000808191819D838C8397FF03C00F969D8365
:102B10008C832C813D8144E0359527954A95E1F7DA
:102B20003D832C83F12CE12C202FA7016C817D812A
:102B300085E094E049D93FEFE31AF30A80E4E81610
:102B4000F10491F71F5F93E0C90ED11C1830A9F66C
:102B500040916F03509170034230510571F138F488
:102B60004130510559F02696E2E10C94982B433000
:102B7000510509F473C144305105A9F708E125E76F
:102B800047E756E068E070E085E090E0F8DA4091D1
:102B90005303509154034115510569F010921A08DE
:102BA0001092190810921C0810921B0870E060E047
:102BB00085E094E025DF5DDED6CF27E34BE764E0D8
:102BC00082E01DDE63E070E07D836C8305E010E051
:102BD00021E0A8016C817D8185E094E0F5D80F5F4C
:102BE0001F4F0D301105A1F7EC81FD813196FD835A
:102BF000EC83EC37F10551F74BE76CE270E082E0D3
:102C000090E0C6DD10921F081092200840EF57E0B8
:102C100066E070E086E190E07EDC11E010931F0832
:102C20001093200895E5892E93E0992EC12CD12C84
:102C30007601C39484E090E09D838C83560191E0FB
:102C4000A91AB1081401260137010EE010E086E050
:102C500090E0E9E0AE16B10411F090E080E04EEEB5
:102C600057E0B8012C813D81281B390BC90153DC89
:102C7000B301A20185E094E0C3DE6BEE77E085E06E
:102C800094E02DDCD1014D915D911D0170E060E07B
:102C90002AE085E094E077DEFFEFAF1ABF0A0A5F13
:102CA0001F4F2FEF421A520A620A720A0C321105A4
:102CB00071F6EC81FD81FC96FD83EC8395E0C90EF5
:102CC000D11CE11CF11CEAE08E0E911C4C815D814F
:102CD0004C37510509F0B2CF40EE57E06EE270E09C
:102CE00080E190E018DC40916D0350916E0370E03C
:102CF00060E082E590E090931A08809319080EE254
:102D000010E010931C0800931B0885E094E078DE27
:102D100046ED57E064E370E080E190E0FCDBC090BA
:102D20006903D0906A03E0906B03F0906C03C701D5
:102D3000B60120EC3BE443E050E00E94F928290171
:102D40003A01C701B60120E13EE040E050E00E94B8
:102D5000F9288CE3882E912CA12CB12CCA01B90141
:102D6000A50194010E94F92869837A838B83392E07
:102D7000262EC701B601A50194010E94F928CA01B7
:102D8000B901A50194010E94F9286C83072F182F1F
:102D90009E83B62E22E530E030931A08209319085E
:102DA000A4E3B0E0B0931C08A0931B0841145104A5
:102DB00059F521103AC06A3020F460E385E094E0D0
:102DC0001BDC2AE04C81502F612F7E8185E094E04E
:102DD000DADD6EE285E094E00FDCC701B60126E0A3
:102DE00030E040E050E00E94F928CA01B9012AE031
:102DF00030E040E050E00E94F928AB01BC012AE03D
:102E000085E094E0C0DDAFCE2AE0B301A20185E009
:102E100094E0B9DD6AE385E094E0EEDBF9E0F215D9
:102E200020F060E385E094E0E7DB2AE049815A8105
:102E30006B81732D85E094E0A6DD6AE385E094E084
:102E4000DBDB99E09B1520F060E385E094E0D4DBC8
:102E50002AE04C81502F612F7E81D2CF23E349E7B6
:102E600066E083E0CCDC08E010E01D830C830FEF0C
:102E700017E064E170E0C8010E9481287C01FF2412
:102E8000582F3DEF3503C0011124A8016C817D81CD
:102E9000805C9F4F40DB8FEFE81AF80A0E0D1F1D74
:102EA000AC81BD811696BD83AC83D89711F75BCEFC
:102EB000B0E0A0E0EEE5F7E10C94862B80916F0383
:102EC00090917003019709F043C015DC20916F03C6
:102ED0003091700303E010E02430310511F002E07E
:102EE00010E0CBE3D3E0CA80E880F980EC0CF11C61
:102EF000C7FCFA94F7FC3AC0F982E882488159810C
:102F0000411558403CF06FEF77E0798368839ADD94
:102F100081958A83239683E0C335D80720F30E94E6
:102F2000D5276C01990FEE08FF080E943009C616DC
:102F3000D706E806F90631F06C257D258E259F25FC
:102F40000E947828C801CDB7DEB7E8E00C94A22B28
:102F50008CE00E941808882309F4C1CFD1D801E081
:102F600010E01093700300936F03B9CF1982188299
:102F700069DD8A83C3CF0F931F93CF93DF93809133
:102F80006F0390917003892B09F04DC000EC13E0A2
:102F90001093310300933003F999FECF80EC93E056
:102FA0000E94A42824EC33E03093310320933003B3
:102FB0006F3472448E44974009F089C0F999FECF6E
:102FC0004AE150E064EC73E085E593E00E948C28D0
:102FD000C0913003D09131036A96D0933103C093EE
:102FE0003003F999FECFCE010E94A9288C012296C8
:102FF000D0933103C093300339D98017910709F07A
:1030000066C042E050E05093340340933303109283
:1030100032033091B403332309F469C063DB1092A7
:10302000540310925303CBE3D3E00E942C2820E0FA
:1030300038E040E050E00E94CD287983688302DDCB
:10304000082F0E942C2822E030E040E050E00E944F
:10305000CD28660F771F881F991F6150710981095C
:103060009109069F602D11246A832396B3E0C3352E
:10307000DB07D8F2109235036DEF7FE08CE696E027
:103080000E9404106DE870E185E696E00E9404104D
:1030900065E870E18EE596E00E94041059E15093D6
:1030A00039037AE2709338039DE490933703B3E1D8
:1030B000B093360310923A0381E090E0909370034E
:1030C00080936F03DF91CF911F910F910895A5E534
:1030D000B3E01AE1FD0111921A95E9F781E090E061
:1030E00090933403809333038093320392CFF2DAC8
:1030F00096CFAAE0B0E0EFE7F8E10C947E2B2FE545
:1031000031E03A872987E985FA854281442309F429
:103110002FC120813181240F311D47FD3A95318324
:103120002083578185819681850F911D57FD9A9542
:1031300097FDFDC096838583E985FA856581768153
:103140006038F6E17F0734F060587641E985FA850A
:1031500076836583E985FA85708537FFEDC047FF83
:10316000F2C0783008F0F4C0E985FA851282108642
:10317000A0911803B0911903139709F4F9C0C090F6
:103180005601D0905701C21AD30A009154011091F0
:10319000550189859A850E9465107C01E985FA852B
:1031A00065817681072E000C880B990B0E94C92936
:1031B00025E33AEF4EE85AE30E94B62A2B013C0180
:1031C0000E9493294B015C01C301B2010E94192B9B
:1031D0009B01AC01505829833A834B835C83B60131
:1031E000DD0C880B990B0E94C9292B013C01B80109
:1031F0006E197F09072E000C880B990B0E94C929B4
:103200006D837E838F839887A3019201C501B401EA
:103210000E94B62A6B017C012D813E814F81588529
:1032200069817A818B819C810E94B62A9B01AC01C5
:10323000C701B6010E942B296B017C0120E030E020
:10324000A9010E94B22A87FD93C0E985FA856085AD
:1032500070E090E080E00E94C92920E030E040E882
:1032600051E40E94B62A9B01AC01C701B6010E943D
:103270008F2987FF7DC0A301920169817A818B81AB
:103280009C810E94B62A2B013C012D813E814F81F9
:103290005885C501B4010E94B62A9B01AC01C30147
:1032A000B2010E942A294B015C0120E030E0A90113
:1032B0000E94B22A18160CF050C020E030E040E81E
:1032C00052E4C501B4010E948F2987FF51C020E05C
:1032D00030E040E85DE3C701B6010E94B62A0E94D3
:1032E0009B29E985FA8560870091500111859091AD
:1032F000530119134DC140915101509152014F5F3B
:103300005F4F50935201409351010160009350016F
:1033100003E010E0E985FA8585819681418566E0C4
:10332000805C944F9ADB01501109A1F721C08058AD
:10333000994EE985FA85FECE2115F8E03F071CF08D
:1033400014160CF40ECF7E5F713918F070E901C0CD
:103350007850E985FA8570870BCF20E030E040E8AF
:1033600052ECC501B4010E94B22A18160CF4AFCF7A
:1033700089859A850A969A878987875D914008F49E
:10338000C2CEA0915D01B0915E011197B0935E0134
:10339000A0935D011A161B060CF4F6C080915B0128
:1033A00090915C016CE070E00E94632B8C010E94A4
:1033B0002C283AE0309FA001319F500D1124415A32
:1033C0005E4F5A83498322E030E040E050E00E94A3
:1033D000CD2820E638E0629FC001639F900D729F68
:1033E000900D1124DC01D097E981FA81B183A0838B
:1033F0000E942C2825E030E040E050E00E94CD28DB
:10340000AB01BC014A5F5F4F6F4F7F4FA981BA810B
:103410008D919C91181619060CF4C6C0B1E0FAE023
:10342000F09F9001F19F300D1124215A3E4F3A83B5
:103430002983B49F802C1124F90182820E942C28B8
:1034400030E4C32ED12CE12CF12CA70196010E946F
:10345000CD28E981FA8164830E942C28A701960176
:103460000E94CD28E981FA819480691963830E94C2
:103470002C2820E836E140E050E00E94CD280E9450
:10348000C92925E33AEF4EE85CE30E94B62A0E9480
:103490009629E981FA81768365830E942C284B0165
:1034A0005C010E942C2822E030E040E050E00E94C5
:1034B000CD286B017C01CC0CDD1CEE1CFF1CF1E067
:1034C000CF1AD108E108F108C501B40121E230E0CA
:1034D00040E050E00E94CD28605F7F4F8F4F9F4FAC
:1034E000C69EC02C1124E981FA81C78210860E94F1
:1034F0002C2828E030E040E050E00E94CD28509198
:103500005A01C52E052E000CDD08EE08FF0831E03B
:103510006C157D058E059F050CF430E04AE0409F58
:10352000F001419FF00D1124E15AFE4F31875150B7
:10353000432F440F450F40935A016C157D058E05AE
:103540009F05A4F16FE774E07093590160935801EF
:1035500080915B0190915C01DC011196B0935C015C
:10356000A0935B01B7FD1396B595A795B595A79563
:10357000B195A195B109A65ABF4FAE31B105CCF0B6
:10358000B0935E01A0935D012A96E0E10C949A2B22
:1035900020914E0130914F012C53310930934F014E
:1035A00020934E010360B2CEBFEF39CF61E674E0E5
:1035B000CBCFAEE1B0E0E4CFAFE0B0E0E2EEFAE1D5
:1035C0000C947C2B0E94A9102091180330911903B0
:1035D0003A8329832130310509F0F5C080914E01ED
:1035E00090914F01803233E093070CF0FDC068ECFE
:1035F00070E00E94632B7727CB01039629813A81E3
:1036000001C0220F8A95EAF7822F8695215090916A
:1036100049012923821B082E000C990B97FF03C038
:1036200091958195910923E030E0261B370B02C06C
:10363000880F991F2A95E2F7E3E0660F771FEA9556
:10364000E1F7861B970B97FD80E010E0EE24EA94EB
:10365000F12CB701681B71098AE00E94C00BB70109
:10366000611B710983E00E94C00B6FEF70E089E07D
:103670000E94C00BE981FA81349709F4F7C22091C6
:10368000560130915701B90154E0759567955A95E7
:10369000E1F77E836D83E0915401F0915501AF0114
:1036A00064E0559547956A95E1F758874F83A7EDF4
:1036B000B1E0BB87AA87EA85FB853381332309F410
:1036C00096C060817181072E000C880B990B0E94B7
:1036D000C92925E33AEF4EE85AE30E94B62A4B0186
:1036E0005C01EA85FB85628170E090E080E00E94E9
:1036F000C92920E030E040E85EE30E94B62A6B0171
:103700007C01EA85FB853480C501B4010E94192B38
:1037100069837A838B839C832F813885B901330F2A
:10372000880B990B0E94C9292B013C0129813A8100
:103730004B815C81C701B6010E94B62A9B01AC0196
:10374000C301B2010E942A290E9496298B01C5015A
:10375000B4010E9493294B015C01ED81FE81BF0100
:10376000FF0F880B990B0E94C9292B013C01A50171
:103770009401C701B6010E94B62A9B01AC01C301A6
:10378000B2010E942B290E9496296B01F2E0CF0E14
:10379000D11C7B0177FF02C0F12CE12CC60121E88E
:1037A000C216D10414F080E890E0E816F906FCF4A3
:1037B000232DA801B70185E094E00E94E40E3FEFBD
:1037C000E31AF30AEBCF89819A81039769F4809118
:1037D000490190914A018031910530F48195880F1B
:1037E000880F805C182F32CF10E080E02FCFAA85A1
:1037F000BB851596BB87AA87A751B34008F45BCF5A
:103800002FE531E03A832983E981FA8152815523FA
:1038100009F4DBC00081118134E0159507953A95D4
:10382000E1F7CF010E9465101C0144E03594279414
:103830004A95E1F7E981FA8165817681072E000CCE
:10384000880B990B0E94C92925E33AEF4EE85AE309
:103850000E94B62A4B015C01E981FA81F185F98762
:103860000E94192B6B017C01E981FA81608570E06F
:1038700090E080E00E94C9296A877B878C879D87BA
:10388000B101032C000C880B990B0E94C9292B0154
:103890003C012A853B854C855D85C701B6010E94A8
:1038A000B62A9B01AC01C301B2010E942A290E94E1
:1038B00096296B017F876E87C501B4010E94932909
:1038C0002B013C01B801012E000C880B990B0E94C2
:1038D000C9294B015C01A30192016A857B858C8516
:1038E0009D850E94B62A9B01AC01C501B4010E94CE
:1038F0002B290E9496295B0136016218730877FE16
:1039000003C07194619471084B01801A910A97FE6B
:1039100003C09194819491088614970444F07F87A2
:103920006E875601922D432C1801092F142DCE8439
:10393000DF84C214D3045CF05A2CDB2C5801052D13
:103940001D2DEE84FF843F862E862E2C3F2C2101D8
:103950006E857F85461A570A6801CA18DB08D7FEAC
:1039600003C0D194C194D108720157FE03C09FEFE8
:10397000E91AF90AF594E794A016B10624F511E0C6
:10398000EE85FF852E163F0604F12985AF01B501AE
:10399000861497041CF0A5016E857F8585E094E070
:1039A0000E94E40EEC18FD08F7FE06C0A10EB11C43
:1039B00017FDBA94E40CF51C4E855F854F5F5F4F91
:1039C0005F874E87DDCF1FEFDBCF89819A810A9613
:1039D0009A838983875D914008F416CFAFE5B1E003
:1039E000BA83A983E981FA817281772309F450C0EF
:1039F000A080B180A4E0B594A794AA95E1F7CF0187
:103A00000E9465104C01B4E095948794BA95E1F753
:103A1000E981FA818581968188589F4F60EF70E037
:103A20000E94632BCB0168E170E00E94632B3C0194
:103A30007724F7E08F9F9001112422563D4FA40177
:103A400043505109B50163507109E981FA81C1847C
:103A500007E0E02E07E085E094E00E94EB0DE981AD
:103A6000FA81C18401E0C0269301220F331F260D85
:103A7000371D2A5A3D4FA40141505109B5016150EB
:103A8000710993E0E92E03E085E094E00E94EB0DDC
:103A900029813A81265F3F4F3A832983275D314050
:103AA00008F4A0CF80914E0190914F019A838983B1
:103AB000181619060CF07BC081E090E010914801C7
:103AC000183014F490E080E0AF80B884A81AB90AE6
:103AD000F090530111E01F25A50143505109C12E5B
:103AE00038E0E32E09E020E533E06D817E8164500B
:103AF000710985E094E00E94EB0DA5014250510947
:103B0000CF2C66E0E62E07E029E433E06D817E816C
:103B10006350710985E094E00E94EB0DA5014150CE
:103B20005109B09147014B0F511DB7FD5A95309186
:103B300046016D817E8161507109630F711D37FDF2
:103B40007A95C12EE4E0EE2E03E026E433E085E032
:103B500094E00E94EB0DE981FA81E83E23E0F20750
:103B600034F5CF016AE070E00E94632BAB01770F60
:103B7000660B770B90914501A90EB11C97FDBA9485
:103B8000AD81BE811597E436F1050CF073C0E3E01A
:103B9000F0E0AE0FBF1FB0931A08A0931908B092BF
:103BA0001C08A0921B0885E094E00E9400158091FB
:103BB0004D0130E020E0882311F022E030E0409118
:103BC00051015091520160914C01062E000C770B6F
:103BD000082E000C990B0E94EE1080915B019091D1
:103BE0005C01892B51F40FE021E34FEF53E068E0D3
:103BF00070E088E290E00E94BF106091180370911D
:103C000019036330710549F50BE02DE445E653E0F7
:103C10006AE170E089E190E00E94BF1050914B0191
:103C2000552321F18091490190914A0123E0969515
:103C300087952A95E1F7817080931F08809320086B
:103C400049E553E068E270E08FE190E00E948B125A
:103C500041E040931F0840932008209118033091C1
:103C600019032230310511F40E9439142F96E2E134
:103C70000C94982BF0E0E0E08CCFCF93DF93809111
:103C80003203882309F455C0209133033091340363
:103C90002130310509F050C040EC53E0509331031E
:103CA00040933003F999FECF4FE452E46EE477E09D
:103CB00080EC93E00E94C528A0913003B0913103BD
:103CC0001496B0933103A0933003F999FECF60911D
:103CD0003003709131034AE150E085E593E00E94A2
:103CE000AE28C0913003D09131036A96D09331034E
:103CF000C09330030E943611F999FECFBC01CE016A
:103D00000E94CA28E0913003F09131033296F0937B
:103D10003103E09330036091B40382E090E00E94AD
:103D2000B72862E070E0709334036093330310921D
:103D30003203DF91CF910895A4ECB3E0C2CFCF93CB
:103D400080916D0390916E03019690936E03809322
:103D50006D03C1E0C093320390DF109252011092C4
:103D6000510110924D0147EF40934C0128EE33E092
:103D700030934F0120934E014093450110924A0128
:103D80001092490160E074E070935701609356010E
:103D9000A0E0B2E0B0935501A09354011092480105
:103DA000C093530134E030935A01EFE5F1E0128201
:103DB0003A9681E0E73DF807D0F310925C0110924B
:103DC0005B0188E790E090935E0180935D01E7EDF1
:103DD000F1E01382359683E0E731F807D0F31092D3
:103DE000170341E050E0509319034093180360E03B
:103DF00080ED91E00E94BB0D10924401CF91089597
:103E0000CF93DF938091180390911903823091052D
:103E100009F4F6C18330910509F4F5C1019709F061
:103E2000A2C1109250011092590110925801A09114
:103E30005B01B0915C011A161B06A4F52091690381
:103E400030916A0340916B0350916C032F5F3F4F99
:103E50004F4F5F4F2093690330936A0340936B0386
:103E600050936C03C0914901D0914A012196D0939F
:103E70004A01C0934901C770DD27CD2B49F4E09179
:103E80005101F09152013196F0935201E0935101AA
:103E900030914C0137FF03C03F5F30934C0141E04C
:103EA0004093320380914E0190914F01883E23E070
:103EB00092072CF4019690934F0180934E0110923B
:103EC0004601109247015091220855FF03C09FEF11
:103ED0009093460156FF05C0609146016F5F609365
:103EE000460157FF03C07FEF7093470154FF05C0A1
:103EF000B0914701BF5FB0934701D0914601F09167
:103F00004701DF02D001112428E0AB2B09F026E0A5
:103F10004091560150915701D202400D511D11247C
:103F2000403451050CF48FC0509357014093560113
:103F30008091560190915701813B974034F060EB9E
:103F400077E07093570160935601A0915401B091AE
:103F50005501F202A00DB11D1124A034B1050CF4DD
:103F600075C0B0935501A093540120915401309134
:103F70005501213B334034F040EB53E05093550161
:103F800040935401C0914801CF5FCF70C093480166
:103F9000D11104C0F11102C01092480184E00E94C6
:103FA0001808882361F0E091530131E0E327E093A2
:103FB000530186EE91E090935901809358015091FE
:103FC0004D01511146C0A0915601B0915701A13445
:103FD000B24034F498E790934D0178EF70934C0120
:103FE000C0915401D0915501C03543E0D4073CF451
:103FF00020914E0130914F01283E334019F4B7EF24
:10400000B0934501C13AD1051CF4D6E0D0934501E7
:1040100070D80E945410C0915001F0914401FC17D7
:1040200049F1C13009F464C0C33009F467C0C1115B
:104030001FC0D0E04091B203D417C0F48D2F0E946E
:10404000B70CDF5FF7CF40E450E06ECFA0E4B0E004
:1040500088CF15162CF66091560170915701603B80
:1040600075400CF4BDCF10924D01B7CF1092B30341
:10407000C09344018091580190915901009741F0FB
:1040800063E021E0863E920709F064E00E94BB0DE8
:10409000E0914E01F0914F011E161F060CF470C006
:1040A000D0E0C0E0409153016BE0CE010E942D159D
:1040B000C65ADF4FC03846E1D407A1F740915101FD
:1040C000509152012AE030E0C9019C012150310990
:1040D000F901EE0FFF1FEB5AFC4F608171816417ED
:1040E000750780F42930310591F489E090E0EDCF37
:1040F00062E085E192E00E94BB0DBACF62E084EFFE
:1041000091E0F9CF8A309105A1F09C010AC0880F97
:10411000991FDC01AB5ABC4F6D937C93211531057F
:1041200099F6E901CC0FDD1FCB5ADC4F5983488348
:10413000C901509354034093530371E0892B09F054
:1041400070E070934B0199DD10924A011092490181
:1041500043E050E0509319034093180361E086E276
:1041600092E00E94BB0D2091180330911903243076
:10417000310509F07AC082E090E0DF91CF91089597
:1041800080915B0190915C011816190664F788E034
:104190000E941808882339F370DD1092350361EA14
:1041A00070E18DE492E00E94041065E970E188E41A
:1041B00092E00E94041032E2309339035AE15093A6
:1041C00038036BE360933703A1E1A09336031092A9
:1041D0003A0322E030E03093190320931803C0E043
:1041E0009091B203C91728F48C2F0E94B70CCF5FAF
:1041F000F7CF1092B3030E94801010924401B3CF06
:104200000E947B13B0CFE0914901F0914A013196B1
:10421000F0934A01E0934901B0914C01B7FF03C00C
:10422000BF5FB0934C010E9479180E945410C09156
:104230004901D0914A01CC33D10508F494CF88E0EC
:104240000E941808811103C0C835D24030F064E0E4
:1042500070E0709319036093180384E00E941808BB
:10426000882309F480CF6BDD7ECF83E090E085CF9B
:104270001F920F920FB60F9211248F939F938091EC
:10428000E1009091E100937F9093E10083FF0FC0E4
:104290001092E90091E09093EB001092EC0092E311
:1042A0009093ED001092AD0398E09093F00082FFA0
:1042B00022C093E09093E9009091F200992319F0C5
:1042C0009AE39093E80090919E03992341F0909196
:1042D0009E03915090939E03911101C05D9A90911D
:1042E000AC03992341F09091AC0391509093AC03AF
:1042F000911101C0289A84FF18C09091E2009E7E1F
:1043000091609093E2008091E1008F7E8093E100C4
:1043100080919F038E7E806180939F039F918F91F8
:104320000F900FBE0F901F90189580FFF7CF8091D0
:10433000E2008E7E80618093E2009091E1009E7E9B
:104340009093E10080919F038E7E8160E5CF1F9264
:104350000F920FB60F921124CF92DF92EF92FF923D
:104360000F931F932F933F934F935F936F937F937D
:104370008F939F93AF93BF93EF93FF93CF93DF936D
:10438000CDB7DEB76C97DEBFCDBF1092E90080914C
:10439000E80083FF25C068E0CE0145960E94060B29
:1043A00002EF0093E8001D8917FF39C0C090E800B4
:1043B000C0FEFCCF212F207609F033C13E894F8902
:1043C000588D6F89F88C311131C0103861F5F0903B
:1043D0009D03F092F1001092F100FEEFF093E800DF
:1043E0006C960FB6F894DEBF0FBECDBFDF91CF91B4
:1043F000FF91EF91BF91AF919F918F917F916F91BD
:104400005F914F913F912F911F910F91FF90EF90EE
:10441000DF90CF900F900FBE0F901F9018959EEFDA
:104420009093E800C7CF1092F100D5CF313059F406
:104430001111D3CF4130510581F680919D038D7FBD
:1044400080939D03CACF333049F41111C6CF413058
:10445000510519F680919D038260F2CF353041F409
:10446000D090E800D0FEFCCF60686093E300B5CF49
:10447000363009F0A8C00B8D1C8D92E01092E90037
:1044800010929B0310929A03F9122EC01092990376
:10449000109298030E94DB0A1F8259E05983FA8226
:1044A00071E07E83B0EAB8872AEF298740919A03AA
:1044B00050919B03475F5F4F5C834B838D831092CA
:1044C000E90010929B0310929A03109399030093B2
:1044D000980349E050E0BE016F5F7F4F80E00E948B
:1044E000BA0A0E94DB0A79CF1093990300939803CC
:1044F0000E948409FC01C280D380C114D10409F454
:1045000052C1D601ED91FC910480F581E02DBE01F0
:104510006B5E7F4FC6010995009709F03FC1F60118
:10452000C084D184EACF33E0F3120EC04F89442314
:1045300009F440C0423061F440E867E081ED9FE05B
:104540000E948D0A811149CF61E26093EB0048CF50
:10455000413029F440E86BE085EC9FE0F1CF433037
:1045600099F70E948409FC01C280D3808E010F5FFD
:104570001F4F7801C114D10479F0D601ED91FC915F
:104580000680F781E02DB801C6010995080F111DBD
:10459000F601C084D184EECFD8011C92F7010190BE
:1045A0000020E9F7BF01615071096E197F0940E0F1
:1045B000C701C6CF6FEA7FE0FB01449150E080E87D
:1045C0000E94BA0A0ACF373009F4BECF383021F43E
:1045D000F1E0F093F10001CF393009F0FECE137015
:1045E00009F0B2CFE6E1F1E081E05191552381F08D
:1045F0008093E90071E07093EB00DF011197CC909C
:10460000C092EC00B6E3B093ED008F5F873069F79E
:104610002EE72093EA001092EA00EF88E092AD03C3
:10462000DCCEEB8CFC8C1092E90010929B03109274
:104630009A03F0929903E0929803D98CD11094C018
:104640003E894D89413A49F4313209F07DCF47E046
:1046500050E065E071E080E0B3CF413209F074CF03
:10466000333269F48F89988DB0E0A0E08093010126
:1046700090930201A0930301B0930401AECE3032B7
:1046800069F4D090E800D2FEFCCF67E085E091E0CD
:104690000E94060B0BEF0093E8009FCE323209F028
:1046A0009CCEFF88F0920C01EEEFFFE765917491CC
:1046B0006B3F7C4D51F1E0E0F8E080910501909175
:1046C0000601A0910701B0910801803B9440A1052B
:1046D000B105F1F450910C0150FD1AC0EE3F8AE093
:1046E000F80791F5A7E7B7E7B183A083F0916000E1
:1046F000F0939C0318E19BE00FB6F894A8951093F3
:1047000060000FBE9093600068CEEEEFFAE0D5CF68
:10471000C080D180A7E7CA16DA0609F05ECEA89558
:1047200070916000786170936000B0919C03B093C9
:104730006000EE3F2AE0F20791F02091FE0A3091EE
:10474000FF0A3183208349CEE080F180B7E7EB1682
:10475000FB0641F2F092FF0AE092FE0AC3CF1092EC
:10476000FF0A1092FE0A39CE0E948409FC010281E0
:1047700013810115110509F4E7CED801ED91FC91E3
:104780000190F081E02DBE016B5E7F4FC80109955D
:10479000811123CEF80100851185EBCF181619067B
:1047A0000CF41BCED1CE11E0F112BDCE63EB7FE055
:1047B00003CF0F920FB68F939F93EF93FF93809148
:1047C0008F038D5F8D3708F08D5780938F03E0E95D
:1047D000F3E080818E4F808391819F4F918382810E
:1047E0008F4F828383818F4F8383E4E9F3E080815D
:1047F0008F5F808381818F4F818382818F4F8283FE
:1048000083818F4F83838FB18F6066991C9B88272C
:104810008F3681F480918E03981B963068F0E0E02B
:10482000F8E087E78083818388E180936000F093DC
:104830006000FFCF90938E03FF91EF919F918F9136
:104840000FBE0F9018951F920F920FB60F92112462
:104850002F933F934F935F936F937F938F939F9388
:10486000AF93BF93EF93FF9380918103882349F027
:1048700020918203E0918303F091840390812927A2
:1048800020833091B303332331F140917D03509164
:104890007E0360917F0370918003452B462B472B4D
:1048A000D1F060917D0370917E0380917F039091A0
:1048B0008003615071098109910960937D037093B0
:1048C0007E0380937F0390938003672B682B692B73
:1048D00011F40E94500DFF91EF91BF91AF919F9104
:1048E0008F917F916F915F914F913F912F910F9099
:1048F0000FBE0F901F9018951F920F920FB60F9238
:1049000011248F939F93AF93BF93EF93FF93809165
:104910007C03882309F452C0809178039091790335
:10492000A0917A03B0917B03892B8A2B8B2BA1F169
:10493000A0918503E0918603F091870380818A2707
:1049400080838091780390917903A0917A03B0914C
:104950007B03181619061A061B069CF4809178032F
:1049600090917903A0917A03B0917B030197A109FB
:10497000B1098093780390937903A0937A03B0935D
:104980007B03FF91EF91BF91AF919F918F910F901A
:104990000FBE0F901F90189510927C03B0916F007E
:1049A000BD7FB0936F00A0918503E0918603F091E5
:1049B00087039081A095A923A083E3CF90918503DD
:1049C000E0918603F0918703A081A927F5CFE5EB5D
:1049D000F3E01382128288EE93E0A0E0B0E08483DB
:1049E0009583A683B78380E291E0918380838FEFE4
:1049F0009FEF95878487E5E0F4E0138212828CE3D1
:104A0000868380E181871086178216861786108A32
:104A1000118A128A10921A081092190810921C0812
:104A200010921B0881E080931D0822E331E031835E
:104A3000208380931F08109220080895789483E0C3
:104A400084BD83E085BD81E080936E00E1E8F0E005
:104A500083E08083E0E881E08083E1E983E0808394
:104A6000E0E981E08083E1EC87E08083E3EC81E0B2
:104A70008083E0EC82E08083E2EC81E08083EAE7FF
:104A800087E08083806880831092AD0310929D033D
:104A900010929F031091D70011601093D70020EA65
:104AA0002093D80039B5306139BD49B5426049BD60
:104AB00009B400FEFDCF0E941D095091D8005F7C13
:104AC00050615093D8006091E000607F6093E000F7
:104AD0007091E1007E7E7093E1009DE09093E20092
:104AE000559A209ACFB7F894A0918803A11127C0B6
:104AF000E1E2FFE0B491E0E4FFE0D491EB2FF0E0DD
:104B0000EE0FFF1FEC50F14FA591B491FC91FD23E6
:104B100021F461E081E10E94130B61E081E10E94D8
:104B2000840B8CB580618CBD1CB510641CBD61E02C
:104B30008FE00E94840B61E080E10E94840B209151
:104B400088032F5F20938803CFBFC9ECDEE0AE015E
:104B5000FE0184914F5F5F4F2296FA016491882392
:104B600019F00E94840BF3CF61E082E00E94130BE6
:104B700061E070E080E090E00E945F0C60E082E025
:104B80000E94130B6AE070E080E090E00E945F0CEE
:104B900061E082E00E94130B61E17FE0FB01E491A0
:104BA000F0E0EE0FFF1FEE5FF04F25913491E0E350
:104BB000FFE05491FB01E491F0E0EE0FFF1FEE5F88
:104BC000F04FA591B4913C91752F709573237C9310
:104BD000E4E1FFE0E491F0E0EE0FFF1FEE5FF04F45
:104BE0008591949190938B0380938A03E3E3FFE094
:104BF000949190938903BCB5BC7FBCBDDDB5D160F9
:104C0000DDBD0E94AC0CECEBFEE014911EBD00007B
:104C10000DB407FEFDCF8EB531963EE0E93CF307BB
:104C2000A1F7C0918A03D0918B03F8812091890369
:104C3000F22BF883409164004160409364006091DE
:104C40006400626060936400509164005068509307
:104C50006400A0916400A064A0936400309165009A
:104C60003160309365000E94990C87FF29C00E9433
:104C7000AC0C35EA3EBD00000DB407FEFDCF8EB58D
:104C8000C0918A03D0918B03788190918903792B0D
:104C9000788370E060E08AE00E94C00B70E060E022
:104CA00083E00E94C00B70E060E089E00E94C00BCE
:104CB000D0916400D062D09364000E94A10CFDCF1B
:104CC0007091B203723091F0E72FF0E0E654F14FAB
:104CD000D4917F5F7093B20361E085E00E94840B02
:104CE000D13009F45FC0D33009F47EC061E086E0C2
:104CF0000E94840B82E090E01FD2882309F49DC0BB
:104D00000E9472134CE340930B0460E160930E0425
:104D100051E050931F085093200810928D03109279
:104D20008C03ECEDFEE0A591B491FD0109953FB730
:104D3000F8948091900390919103A0919203B09187
:104D400093033FBF70911704772391F0D0910F0424
:104D5000282F2D1B2093180440910C0450910D0412
:104D60004F5F5F4F50930D0440930C041092170453
:104D7000409113045091140460911504709116042D
:104D800084179507A607B7070CF05AC0481B423096
:104D900010F00E94A10CA0E0B0E0AB2B41F20E9409
:104DA0000000C5CF1092800010928100E091810038
:104DB000E860E09381001091810011601093810000
:104DC000E5E1FFE0E491F0E0EE0FFF1FEE5FF04F52
:104DD000259134913093870320938603E4E3FFE029
:104DE000F491F093850382CF10929000109291007D
:104DF00080919100886080939100909191009160E2
:104E000090939100E5E1FFE0E491F0E0EE0FFF1FE9
:104E1000EE5FF04FC591D491D0938403C093830388
:104E2000E4E3FFE0B491B09382036CE380E00E947E
:104E3000DA0C80E00E94B70C59CF0E946A1362CF4F
:104E400010910E04AC01BD01410F511D611D711D7A
:104E50004093130450931404609315047093160444
:104E600080930F0490931004A0931104B093120444
:104E700081E08093170490912208909321080E946A
:104E8000990C8093220860918C0370918D0316E039
:104E9000169FF001179FF00D1124E252F14FA591DA
:104EA000B491FD010995EC0120918C0330918D03A3
:104EB000129FF001139FF00D1124E052F14F459124
:104EC0005491FA010995B0911904BEBDAAE1B4E06C
:104ED00089E198E0FD910DB407FEFDCFFEBD8A1774
:104EE0009B07C1F70DB407FEFDCF60918C03709155
:104EF0008D03C617D70709F44ECFD0938D03C09307
:104F00008C0356E05C9FF0015D9FF00D1124E4528C
:104F1000F14FC591D491FE0109953DCF8F929F929B
:104F2000AF92BF92CF92DF92EF92FF92CF93DF9337
:104F3000EC01688179818A819B8161157105810508
:104F4000910521F464E279ED8BE597E02DE133EFF3
:104F500041E050E022D149015A019B01AC01A7EA8E
:104F6000B1E437D16B017C01ACEEB4EFA501940143
:104F70003CD1DC01CB018C0D9D1DAE1DBF1DB7FFCB
:104F800003C00197A109B04888839983AA83BB8392
:104F90009F77DF91CF91FF90EF90DF90CF90BF9000
:104FA000AF909F908F900895B9CF8DE091E0B6CFEC
:104FB000B0E0A0E080930D0190930E01A0930F014B
:104FC000B093100108958F929F92AF92BF92CF92AB
:104FD000DF92EF92FF92CF93DF93EC0168817981AA
:104FE0008A819B81611571058105910521F464E237
:104FF00079ED8BE597E02DE133EF41E050E0CDD046
:1050000049015A019B01AC01A7EAB1E4E2D06B016E
:105010007C01ACEEB4EFA5019401E7D0C60ED71E1B
:10502000E81EF91EF7FE06C081E0C81AD108E108A3
:1050300080E8F80AC882D982EA82FB82C701B601F9
:105040009F77DF91CF91FF90EF90DF90CF90BF904F
:10505000AF909F908F9008958F929F92AF92BF9242
:10506000CF92DF92EF92FF92609111017091120145
:1050700080911301909114016115710581059105CD
:1050800021F464E279ED8BE597E02DE133EF41E027
:1050900050E083D049015A019B01AC01A7EAB1E479
:1050A00098D06B017C01ACEEB4EFA50194019DD0CA
:1050B000C60ED71EE81EF91EF7FE06C081E0C81A0C
:1050C000D108E10880E8F80AC0921101D0921201DB
:1050D000E0921301F0921401C701B6019F77FF908F
:1050E000EF90DF90CF90BF90AF909F908F900895FA
:1050F0006093110170931201809313019093140136
:105100000895FC010590615070400110D8F780951A
:1051100090958E0F9F1F0895DC01CB01FC01F9993A
:10512000FECF06C0F2BDE1BDF89A319600B40D92F3
:1051300041505040B8F70895F999FECF92BD81BD16
:10514000F89A992780B50895A6E1B0E044E050E0D0
:10515000E5CFA8E1B0E042E050E0E0CFDC01CB01D8
:1051600002C02D9105D041505040D8F70895262F08
:10517000F999FECF1FBA92BD81BD20BD0FB6F8943C
:10518000FA9AF99A0FBE01960895242FF1DF252F80
:10519000EFDF00C0ECDF272FEBCF052E97FB16F4D7
:1051A00000940FD057FD05D024D007FC02D046F460
:1051B00008C050954095309521953F4F4F4F5F4F18
:1051C000089590958095709561957F4F8F4F9F4F73
:1051D000089531D0A59F900DB49F900DA49F800D90
:1051E000911D11240895B7FFF4CFF3DF821B930BB9
:1051F0000895A1E21A2EAA1BBB1BFD010DC0AA1F18
:10520000BB1FEE1FFF1FA217B307E407F50720F02F
:10521000A21BB30BE40BF50B661F771F881F991FAA
:105220001A9469F760957095809590959B01AC01F3
:10523000BD01CF010895A29FB001B39FC001A39FFC
:10524000700D811D1124911DB29F700D811D1124BF
:10525000911D08955058BB27AA270ED038C101D1FF
:1052600030F006D120F031F49F3F11F41EF4F6C067
:105270000EF4E095E7FBECC0E92F4BD180F3BA17B1
:10528000620773078407950718F071F49EF563C1F0
:105290000EF4E0950B2EBA2FA02D0B01B901900151
:1052A0000C01CA01A0011124FF27591B99F0593F95
:1052B00050F4503E68F11A16F040A22F232F342FDD
:1052C0004427585FF3CF469537952795A795F0402B
:1052D0005395C9F77EF41F16BA0B620B730B840B40
:1052E000BAF09150A1F0FF0FBB1F661F771F881FF8
:1052F000C2F70EC0BA0F621F731F841F48F4879550
:1053000077956795B795F7959E3F08F0B3CF93953E
:10531000880F08F09927EE0F97958795089574D018
:1053200008F481E00895ACD0E395E2C004D068941D
:10533000B11112C10895F5D088F09F5790F0B92FA0
:105340009927B751A0F0D1F0660F771F881F991FDA
:105350001AF0BA95C9F712C0B13081F0FCD0B1E0B3
:105360000895F9C0672F782F8827B85F39F0B93FC3
:10537000CCF3869577956795B395D9F73EF49095DC
:105380008095709561957F4F8F4F9F4F0895E8945A
:1053900009C097FB3EF490958095709561957F4F7D
:1053A0008F4F9F4F9923A9F0F92F96E9BB2793952B
:1053B000F695879577956795B795F111F8CFFAF43B
:1053C000BB0F11F460FF1BC06F5F7F4F8F4F9F4F6C
:1053D00016C0882311F096E911C0772321F09EE8CA
:1053E000872F762F05C0662371F096E8862F70E030
:1053F00060E02AF09A95660F771F881FDAF7880F0A
:105400009695879597F90895990F0008550FAA0B5F
:10541000E0E8FEEF16161706E807F907C0F01216C7
:105420001306E407F50798F0621B730B840B950BCA
:1054300039F40A2661F0232B242B252B21F408951F
:105440000A2609F4A140A6958FEF811D811D0895BC
:1054500097F99F6780E870E060E008959FEF80EC27
:10546000089500240A9416161706180609060895CA
:1054700000240A9412161306140605060895EECFAA
:1054800050D0E8F3E894E0E0BB279F57F0F02AED16
:105490003FE049EC06C0EE0FBB0F661F771F881F69
:1054A00028F0B23A62077307840728F0B25A620BF9
:1054B000730B840BE3959A9572F7803830F49A95C4
:1054C000BB0F661F771F881FD2F79048BAC0092EFE
:1054D0000394000C11F4882352F0BB0F40F4BF2B4F
:1054E00011F460FF04C06F5F7F4F8F4F9F4F08958F
:1054F000EF93E0FF06C0A2EA2AED3FE049EC5FEB44
:10550000BBDEE5DF0F90039401FC9058ECEAF0E07D
:10551000A4C057FD9058440F551F59F05F3F71F0DC
:105520004795880F97FB991F61F09F3F79F087950A
:105530000895121613061406551FF2CF4695F1DF93
:1055400008C0161617061806991FF1CF8695710523
:10555000610508940895E894BB2766277727CB0157
:1055600097F9089551DF08F48FEF08950BD0AFCF6E
:1055700078DF28F07DDF18F0952309F069CF6ECF32
:105580001124EACFC6DFA0F3959FD1F3950F50E029
:10559000551F629FF001729FBB27F00DB11D639FE5
:1055A000AA27F00DB11DAA1F649F6627B00DA11D8B
:1055B000661F829F2227B00DA11D621F739FB00D31
:1055C000A11D621F839FA00D611D221F749F3327A1
:1055D000A00D611D231F849F600D211D822F762F3A
:1055E0006A2F11249F5750408AF0E1F088234AF037
:1055F000EE0FFF1FBB1F661F771F881F9150504083
:10560000A9F79E3F510570F023CFA6CF5F3FECF383
:10561000983EDCF3869577956795B795F795E7956E
:105620009F5FC1F7FE2B880F911D9695879597F97F
:1056300008959F9325DF0F9007FCEE5F59CF9F3FA2
:1056400031F0915020F4879577956795B795880F3D
:10565000911D9695879597F908959F938F937F93C2
:105660006F93FF93EF939B01AC0180DFEF91FF916C
:1056700005D02F913F914F915F9178CFDF93CF93DA
:105680001F930F93FF92EF92DF927B018C0168943E
:1056900005C0DA2EEF0176DFFE01E894A591259191
:1056A000359145915591AEF3EF01E6DDFE0197018D
:1056B000A801DA9479F7DF90EF90FF900F911F9196
:1056C000CF91DF91089597FB072E16F4009406D032
:1056D00077FD08D048D007FC05D03EF49095819521
:1056E0009F4F0895709561957F4F0895EE0FFF1FAE
:1056F0000590F491E02D09942F923F924F925F9282
:105700006F927F928F929F92AF92BF92CF92DF92D1
:10571000EF92FF920F931F93CF93DF93CDB7DEB736
:10572000CA1BDB0B0FB6F894DEBF0FBECDBF0994CA
:105730002A88398848885F846E847D848C849B8421
:10574000AA84B984C884DF80EE80FD800C811B812F
:10575000AA81B981CE0FD11D0FB6F894DEBF0FBE5E
:10576000CDBFED010895AA1BBB1B51E107C0AA1FC5
:10577000BB1FA617B70710F0A61BB70B881F991FF2
:105780005A95A9F780959095BC01CD010895F8949C
:02579000FFCF49
:1057920001FFFFFFFF00E100000000000001000028
:1057A200000100000000C180810000000000000034
:1057B200050A9809270A1C0A450A2A0A360A00001D
:0A57C20000004D11760CC513C4134E
:00000001FF
